BL51 BANKED LINKER/LOCATER V6.05                                                        07/15/2014  17:11:25  PAGE 1


BL51 BANKED LINKER/LOCATER V6.05, INVOKED BY:
C:\KEIL\C51\BIN\BL51.EXE dingshiqi.obj TO dingshiqi RAMSIZE (256)


MEMORY MODEL: SMALL


INPUT MODULES INCLUDED:
  dingshiqi.obj (DINGSHIQI)
  C:\KEIL\C51\LIB\C51S.LIB (?C_STARTUP)
  C:\KEIL\C51\LIB\C51S.LIB (?C?UIDIV)
  C:\KEIL\C51\LIB\C51S.LIB (?C?SLCMP)


LINK MAP OF MODULE:  dingshiqi (DINGSHIQI)


            TYPE    BASE      LENGTH    RELOCATION   SEGMENT NAME
            -----------------------------------------------------

            * * * * * * *   D A T A   M E M O R Y   * * * * * * *
            REG     0000H     0008H     ABSOLUTE     "REG BANK 0"
            DATA    0008H     000BH     UNIT         _DATA_GROUP_
            DATA    0013H     0009H     UNIT         ?DT?DINGSHIQI
            IDATA   001CH     0001H     UNIT         ?STACK

            * * * * * * *   C O D E   M E M O R Y   * * * * * * *
            CODE    0000H     0003H     ABSOLUTE     
                    0003H     0008H                  *** GAP ***
            CODE    000BH     0003H     ABSOLUTE     
            CODE    000EH     00DDH     UNIT         ?PR?MAIN?DINGSHIQI
            CODE    00EBH     00DDH     UNIT         ?PR?_DISPLAY?DINGSHIQI
            CODE    01C8H     006BH     UNIT         ?C?LIB_CODE
            CODE    0233H     0024H     UNIT         ?PR?_DELAY?DINGSHIQI
            CODE    0257H     001BH     UNIT         ?PR?INIT?DINGSHIQI
            CODE    0272H     0010H     UNIT         ?CO?DINGSHIQI
            CODE    0282H     000CH     UNIT         ?C_C51STARTUP
            CODE    028EH     0009H     UNIT         ?PR?TIMER0?DINGSHIQI



OVERLAY MAP OF MODULE:   dingshiqi (DINGSHIQI)


SEGMENT                          DATA_GROUP 
  +--> CALLED SEGMENT          START    LENGTH
----------------------------------------------
?C_C51STARTUP                  -----    -----
  +--> ?PR?MAIN?DINGSHIQI

?PR?MAIN?DINGSHIQI             -----    -----
  +--> ?PR?INIT?DINGSHIQI
  +--> ?PR?_DISPLAY?DINGSHIQI

?PR?_DISPLAY?DINGSHIQI         0008H    000BH
  +--> ?CO?DINGSHIQI
  +--> ?PR?_DELAY?DINGSHIQI

BL51 BANKED LINKER/LOCATER V6.05                                                      07/15/2014  17:11:25  PAGE 2




SYMBOL TABLE OF MODULE:  dingshiqi (DINGSHIQI)

  VALUE           TYPE          NAME
  ----------------------------------

  -------         MODULE        DINGSHIQI
  C:0000H         SYMBOL        _ICE_DUMMY_
  D:0080H         PUBLIC        P0
  D:0090H         PUBLIC        P1
  D:00A0H         PUBLIC        P2
  D:00B0H         PUBLIC        P3
  B:00A8H.7       PUBLIC        EA
  C:0272H         PUBLIC        table
  D:00A8H         PUBLIC        IE
  C:0239H         PUBLIC        _delay
  D:00B8H         PUBLIC        IP
  C:000EH         PUBLIC        main
  B:00A0H.6       PUBLIC        dula
  B:00A0H.7       PUBLIC        wela
  D:0098H         PUBLIC        SCON
  D:0089H         PUBLIC        TMOD
  D:0088H         PUBLIC        TCON
  C:0257H         PUBLIC        init
  D:0013H         PUBLIC        temp
  D:0015H         PUBLIC        aa
  B:00A8H.1       PUBLIC        ET0
  D:008CH         PUBLIC        TH0
  D:008AH         PUBLIC        TL0
  C:028EH         PUBLIC        timer0
  D:0016H         PUBLIC        miao0
  D:0017H         PUBLIC        miao1
  D:00C8H         PUBLIC        T2CON
  D:0018H         PUBLIC        fen0
  D:0019H         PUBLIC        fen1
  D:001AH         PUBLIC        shi0
  D:001BH         PUBLIC        shi1
  C:00EBH         PUBLIC        _display
  D:00D0H         PUBLIC        PSW
  -------         PROC          MAIN
  C:000EH         LINE#         16
  C:000EH         LINE#         17
  C:000EH         LINE#         18
  C:0011H         LINE#         19
  C:0011H         LINE#         20
  C:0011H         LINE#         21
  C:001AH         LINE#         22
  C:001AH         LINE#         23
  C:001CH         LINE#         24
  C:0024H         LINE#         25
  C:0037H         LINE#         26
  C:0037H         LINE#         27
  C:003BH         LINE#         28
  C:003BH         LINE#         29
  C:0051H         LINE#         30
  C:005FH         LINE#         31
BL51 BANKED LINKER/LOCATER V6.05                                                      07/15/2014  17:11:25  PAGE 3


  C:0082H         LINE#         32
  C:0090H         LINE#         33
  C:00B9H         LINE#         34
  C:00C7H         LINE#         35
  C:00C7H         LINE#         36
  C:00E8H         LINE#         37
  -------         ENDPROC       MAIN
  C:0233H         SYMBOL        L?0020
  -------         PROC          L?0019
  -------         ENDPROC       L?0019
  C:0233H         SYMBOL        L?0020
  -------         PROC          _DELAY
  D:0006H         SYMBOL        z
  -------         DO            
  D:0006H         SYMBOL        x
  D:0004H         SYMBOL        y
  -------         ENDDO         
  C:0239H         LINE#         40
  C:0239H         LINE#         41
  C:0239H         LINE#         43
  C:0242H         LINE#         44
  C:0256H         LINE#         45
  -------         ENDPROC       _DELAY
  -------         PROC          _DISPLAY
  D:0007H         SYMBOL        shi1
  D:0009H         SYMBOL        shi0
  D:0002H         SYMBOL        fen1
  D:000DH         SYMBOL        fen0
  D:000FH         SYMBOL        miao1
  D:0011H         SYMBOL        miao0
  C:00EBH         LINE#         47
  C:00EFH         LINE#         48
  C:00EFH         LINE#         49
  C:00F1H         LINE#         50
  C:00F8H         LINE#         51
  C:00FAH         LINE#         53
  C:00FDH         LINE#         54
  C:00FFH         LINE#         56
  C:0102H         LINE#         57
  C:0102H         LINE#         58
  C:0105H         LINE#         60
  C:0107H         LINE#         61
  C:0117H         LINE#         62
  C:0119H         LINE#         64
  C:011CH         LINE#         66
  C:011EH         LINE#         67
  C:0121H         LINE#         68
  C:0121H         LINE#         69
  C:0124H         LINE#         71
  C:0126H         LINE#         72
  C:0129H         LINE#         73
  C:012BH         LINE#         75
  C:012EH         LINE#         77
  C:0130H         LINE#         78
  C:0133H         LINE#         79
  C:0133H         LINE#         80
  C:0136H         LINE#         82
BL51 BANKED LINKER/LOCATER V6.05                                                      07/15/2014  17:11:25  PAGE 4


  C:0138H         LINE#         83
  C:0146H         LINE#         84
  C:0148H         LINE#         86
  C:014BH         LINE#         88
  C:014DH         LINE#         89
  C:0150H         LINE#         90
  C:0150H         LINE#         91
  C:0153H         LINE#         94
  C:0155H         LINE#         95
  C:0165H         LINE#         96
  C:0167H         LINE#         97
  C:016AH         LINE#         98
  C:016CH         LINE#         99
  C:016FH         LINE#         100
  C:016FH         LINE#         101
  C:0172H         LINE#         103
  C:0174H         LINE#         104
  C:0177H         LINE#         105
  C:0179H         LINE#         107
  C:017CH         LINE#         109
  C:017EH         LINE#         110
  C:0181H         LINE#         111
  C:0181H         LINE#         112
  C:0184H         LINE#         114
  C:0186H         LINE#         115
  C:0196H         LINE#         116
  C:0198H         LINE#         118
  C:019BH         LINE#         120
  C:019DH         LINE#         121
  C:01A0H         LINE#         122
  C:01A0H         LINE#         123
  C:01A3H         LINE#         126
  C:01A5H         LINE#         127
  C:01B5H         LINE#         128
  C:01B7H         LINE#         130
  C:01BAH         LINE#         132
  C:01BCH         LINE#         133
  C:01BFH         LINE#         134
  C:01C1H         LINE#         135
  -------         ENDPROC       _DISPLAY
  -------         PROC          INIT
  C:0257H         LINE#         138
  C:0257H         LINE#         139
  C:0257H         LINE#         140
  C:0259H         LINE#         141
  C:025BH         LINE#         142
  C:0261H         LINE#         143
  C:0264H         LINE#         144
  C:0267H         LINE#         145
  C:026AH         LINE#         146
  C:026CH         LINE#         147
  C:026EH         LINE#         148
  C:0271H         LINE#         150
  -------         ENDPROC       INIT
  -------         PROC          TIMER0
  C:028EH         LINE#         152
  C:028EH         LINE#         154
BL51 BANKED LINKER/LOCATER V6.05                                                      07/15/2014  17:11:25  PAGE 5


  C:0291H         LINE#         155
  C:0294H         LINE#         156
  C:0296H         LINE#         157
  -------         ENDPROC       TIMER0
  -------         ENDMOD        DINGSHIQI

  -------         MODULE        ?C?UIDIV
  C:01C8H         PUBLIC        ?C?UIDIV
  -------         ENDMOD        ?C?UIDIV

  -------         MODULE        ?C?SLCMP
  C:021DH         PUBLIC        ?C?SLCMP
  -------         ENDMOD        ?C?SLCMP

Program Size: data=29.0 xdata=0 code=655
LINK/LOCATE RUN COMPLETE.  0 WARNING(S),  0 ERROR(S)
